:020000040800F2
:1000000000070020F101000805290008A1280008C8
:10001000E1280008A1280008C1280008F301000811
:10002000F3010008F3010008F3010008513C000847
:10003000F3010008F3010008F3010008F3010008D0
:10004000F3010008F3010008F3010008F3010008C0
:10005000F3010008F3010008054B00082D4B0008D0
:10006000554B00087D4B0008A54B0008F301000824
:10007000F3010008F3010008F3010008F301000890
:10008000F3010008F3010008F30100081D2800082F
:100090004928000875280008F3010008CD4B000826
:1000A000F3010008F3010008F3010008F301000860
:1000B000C94C0008F3010008F3010008F30100082F
:1000C000F3010008F3010008F3010008F301000840
:1000D000F3010008F3010008F3010008F301000830
:1000E000414C0008F3010008F3010008F301000887
:1000F000F3010008F3010008F3010008F301000810
:10010000F3010008F3010008F3010008F3010008FF
:10011000F3010008F3010008F3010008F3010008EF
:10012000F3010008F3010008F3010008F3010008DF
:10013000F3010008F3010008F3010008F3010008CF
:10014000F3010008F3010008F3010008F3010008BF
:10015000F3010008F3010008F3010008F3010008AF
:10016000F3010008F3010008F3010008F30100089F
:10017000F3010008F3010008F3010008F30100088F
:10018000F3010008F3010008F3010008F30100087F
:10019000F3010008F3010008F3010008F30100086F
:1001A000F3010008F3010008F3010008F30100085F
:1001B000F3010008F3010008F3010008F30100084F
:1001C000F3010008F3010008F3010008F30100083F
:1001D000F3010008F3010008F3010008F30100082F
:1001E000FD110008000000000000000000000000F9
:1001F00002E000F000F8FEE772B6374880F30888A6
:10020000364880F3098836483649086040F20000D5
:10021000CCF200004EF63471CEF200010860BFF35C
:100220004F8FBFF36F8F40F20000C0F2F0004EF628
:100230008851CEF200010860BFF34F8FBFF36F8F7C
:100240004FF00000E1EE100A4EF63C71CEF20001D4
:100250000860062080F31488BFF36F8F04F042FA21
:1002600004F02CFB4FF055301F491B4A91423CBF14
:1002700041F8040BFAE71D49184A91423CBF41F886
:10028000040BFAE71A491B4A1B4B9A423EBF51F82E
:10029000040B42F8040BF8E700201849184A914271
:1002A0003CBF41F8040BFAE704F020FA04F00CFB21
:1002B000144C154DAC4203DA54F8041B8847F9E797
:1002C00000F042F8114C124DAC4203DA54F8041B12
:1002D0008847F9E704F008BA00070020002300204F
:1002E0000000000808ED00E00001002000070020E9
:1002F00028510008002300208023002080230020B4
:10030000604D0020E0010008E4010008E40100085D
:10031000E40100082DE9F04F2DED108AC1F80CD052
:10032000C3689D46BDEC108ABDE8F08F002383F3BF
:1003300011882846A047002003F0F4FDFEE703F0F3
:1003400079FD00DFFEE70000F8B500F05FFF04F084
:100350005DF9064604F0B2F90746A8B92C4B9E4257
:100360002BD001339E422BD026F0FF02294B9A421C
:1003700003D0054641F2883408E0F0B200F042FEB6
:100380003D4642F2107401E00546002400F040FEB4
:1003900008B10024254601F0E3FAA0B941F2883300
:1003A0009C4216D017B11C4B9E4216D1002004F07F
:1003B00039F9BDB900F0A6FE26E005460024E5E7C0
:1003C00000240125E2E7032000F030F80024254650
:1003D000E8E74FF47A740125E4E704F067F90024B4
:1003E0002546E3E700F040F8E4E700F0DDFE4FF4D7
:1003F0007A7003F09FFD002CF7D002F08BFA401BBF
:10040000A042F2D900F030F802F084FA0546F2E793
:10041000010007B0000008B0263A09B0302383F38A
:100420001188854680F308880847704708B50C4B4B
:100430001870032806D8DFE800F00A06020E022032
:1004400000F050FF08BD022000F042FFFAE7054B24
:1004500000225A60F6E7034B00225A60F2E700BF21
:10046000802300208423002008B501F079FA034698
:1004700068B9072B0FD89A0002F1006202F58032AA
:100480001268B2F1FF3F05D00133DBB2F1E7032080
:10049000FFF7CCFF08BD174B5A68013B9A42F9D9C8
:1004A000154B9B6803F1006303F580339A42F1D248
:1004B00004F0CEF804F0E0F8002000F0C3FE0220C3
:1004C000FFF7B4FF0D4B1A6C00221A64196E1A66FE
:1004D000196E596C5A64596E5A665B6E72B6054B4A
:1004E0004FF0E022C2F8083D59681868FFF796FF00
:1004F000D0E700BF000001080023002000380240C0
:10050000094A136899B21B0C49F2690000FB0133D8
:100510001360064B186882B2000C44F2506101FB74
:100520000200186080B270471823002014230020B6
:1005300010B50446FFF7E4FFB0FBF4F304FB13002F
:1005400080B210BD10B40346002202604260826097
:10055000C260044C07CC186059609A605DF8044B87
:10056000704700BF107AFF1F70B50E4614461D4637
:1005700002F078FE60B9022D33D1012C01D00020A9
:1005800030E019A3D3E90023C6E90023012029E0C4
:10059000282C1FD00CD8012C15D0052C06D114A363
:1005A000D3E90023C6E9002301201BE0002019E065
:1005B000302C06D110A3D3E90023C6E90023012083
:1005C00010E000200EE00EA3D3E90023C6E90023CB
:1005D000012007E00CA3D3E90023C6E90023012092
:1005E00000E0002070BD00BF401DA12026812A0B25
:1005F000F017304A39059E5678F6339F93CACD8D51
:100600009E6AC421818A46EE26417272DF25D7B7E1
:1006100070B58AB006460D4602F07CF904464FF4E8
:10062000C870FFF785FF044404F51674174B1C606F
:10063000EB7E23B9164B00221A700AB070BD05A9D3
:10064000284600F091FF0028F7D101A8FFF77AFFB4
:100650009DF81640224601A90DF1170004F0C6FBD3
:1006600048B90F2C0BD80A4B1C70084A1368A3F525
:1006700016731360E1E7064B00221A70DDE79DF860
:100680001410304602F0E6FDD7E700BFA03300208B
:100690009D3300202DE9F043ADF5517D80460E4697
:1006A0000DF5E2790027719740F27512394672A86C
:1006B00000F036FE0EAC4FF4C4723946204600F00E
:1006C0002FFE02F027F92F4BA3FB003080092E4BA1
:1006D000186093E8070084E8070002232374677416
:1006E0000DF15A00FFF72EFF042384F820306E230B
:1006F00084F821300DF1180C244D0FCDACE80F001B
:1007000095E80F00ACE80700ACF800301D2384F832
:1007100032310DF1180CBCE80F00CDF86B01CDF8AB
:100720006F11CDF87321CDF87731BCE80700CDF813
:100730007B01CDF87F11CDF883219CF800308DF836
:10074000873101224946204600F03EFE80B20590E6
:10075000CDF810900397B37E029306F1190301932D
:100760000123009305A3D3E90023F17E404602F064
:100770002FFE0DF5517DBDE8F08300BF9E6AC421B8
:10078000818A46EED34D62108C230020D84E00089B
:10079000F0B5FDB006460D462B4B1C7A6CBB07A985
:1007A000284600F025FF002845D19DF81D70C82F70
:1007B00041D84FF4A6620021234800F0B1FD032C7C
:1007C0000AD82202204B4FF48A7101FB0433C3F88C
:1007D000E4200134E4B2F2E71B4C3A460DF11E016D
:1007E00004F1090000F088FDE219002353729DF81E
:1007F0001C3023720BB9EA7E2272812200213AA8B2
:1008000000F08EFD5BAC012221463AA800F02CFFDF
:1008100080B20590049400230393AB7E029305F10C
:10082000190301932823009305A3D3E90023E97E4C
:10083000304602F0CDFD7DB0F0BD00BFAFF30080CB
:1008400026417272DF25D7B7B0440020134BB3F8AE
:100850002C35834200D9704710B50446002100F0C2
:100860001BFD01340D4BA3F82C450C4BB3F82C05A4
:1008700000F0F6FC88B1094BB3F82C0500F002FD3E
:1008800058B9064C0021B4F82C0500F005FDB4F869
:100890002C350133A4F82C35E7E710BDB044002017
:1008A0002DE9F041F0B00646274C94F8D8304FF4CB
:1008B0008A7505FB004585F8DC30002785F8E8706F
:1008C000D82239463AA800F02BFD04F10908404629
:1008D00000F01CFDC2B28DF8F020D5F8E4303A9358
:1008E0003B9741460DF1F10000F006FD06AD0122F7
:1008F00029463AA800F0E2FE80B205900495012353
:1009000003930823029304F1D80301933023009347
:100910000BA3D3E90023217A0C4802F059FDB84219
:1009200003DC002070B0BDE8F08101F0F3FF4FF46C
:100930008A7202FB0646C6F8E0000120F2E700BF1B
:1009400078F6339F93CACD8DB0440020A4330020A5
:1009500038B501F0DFFF0546002408E00532B3EBAF
:10096000420F02D3FFF79CFFF8B10134E4B2032C2D
:100970001BD80E4B93F8D900204400F003004FF42D
:100980008A7202FB003393F8E830002BEDD1074B5D
:1009900002FB0033D3F8E030002BE3D0EB1A034A1C
:1009A0001268F92ADAD8FA22D8E738BDB044002014
:1009B000F0B58FB000230A938DF834308DF83530C0
:1009C0000B930C9300242746002C46D101238DF86D
:1009D0000C3000238DF80D3041F2D80204FB02F2F6
:1009E000204955185258966800200021CDE9000191
:1009F0000DF10D0203A92846B0479DF80C604EB3D7
:100A0000194A536983F48053536100230693079373
:100A10000893099341F2D80304FB03F3114AD35816
:100A20005F690DF10E0304AA0AA92846B84707AB6F
:100A30000BAA92E8030083E803009DF834308DF898
:100A400024300A9B0693DDE9042306A9074802F037
:100A5000C7FE37460134E4B2B6E7002FB2D10FB07B
:100A6000F0BD00BFD833002000080240A4330020AE
:100A700010B586B0BDF828400494099C03949DF8F5
:100A8000204002940193009202460B46024802F075
:100A90003FFC06B010BD00BFA433002010B58AB0E3
:100AA000244802F0DFFB08B10AB010BD01F032FFAC
:100AB000214B1B689842F7D301F02CFF04464FF4FA
:100AC000C870FFF735FD044404F516741A4B1C601A
:100AD00000238DF82030194B1B7813B901238DF8B2
:100AE000203004A8FFF72EFD144B1978C1F1100433
:100AF000E4B2062C00D90624224604AB19440DF1B9
:100B0000210000F0F9FB0134029408AB0193182393
:100B100000930B4B012205A1D1E90001FFF7A8FFCB
:100B2000064B00221A70BFE7AFF30080401DA120E2
:100B300026812A0BA4330020A03300209D330020FF
:100B40009C33002010B586B001F0E4FE0F4BA3FBF0
:100B500000239B090E48036004AC0122214600F0EB
:100B6000DBFC80B20290019418230093094B40F201
:100B7000551204A1D1E90001FFF77AFF06B010BDBC
:100B8000AFF30080F1C6A7C1D068080FD34D621043
:100B90008C230020E449002010B502460B46094C86
:100BA000204602F04DFC204602F05CFB38B1064BBB
:100BB0001B7A2BB10322054B5A71FFF7C3FF10BDFF
:100BC0000222F8E7A4330020B04400208C23002048
:100BD000012800D0704738B54FF6FF73994200D016
:100BE00038BD0025084C002D07DB204601F0BCF97C
:100BF00004F586541834013DF5E7044A0449002001
:100C000004F0A4F8ECE700BFD8330020204A00200D
:100C1000150C000838B50F4C0F4B9C4219D0A4F5A9
:100C20008653A3F118040D4A43F8182C41F25C03D3
:100C3000E21812793AB9E5582DB1284600F09EFE27
:100C4000284604F089F804F58250083000F096FE3A
:100C5000E2E738BDB0440020D8330020384F000808
:100C6000F0B587B0254802F0DFFB002839D00446F4
:100C7000002302938DF814308DF8153003930493FC
:100C8000027B8DF8142003AA4068A16803C2226881
:100C900042F0004202921D461C46D5B941F2D803EB
:100CA00005FB03F3164A9E189B581F6901F036FE98
:100CB000144A82184FF00003009341F1000302A987
:100CC0003046B8470028C8BF44F001040135EDB2F2
:100CD000E3E744B90C4B1B78072B0BD801330A4AC6
:100CE000137007B0F0BD054802F0A2FB064B0022CE
:100CF0001A70B7E7014802F09BFBF2E7A43300202B
:100D0000D833002040420F00E5490020CA7E9B4BAB
:100D10001B7A9A4240F031812DE9F04700AF084636
:100D20000024032C0CD8954B4FF48A7202FB043339
:100D300093F8DC20437E9A4207D00134E4B2F0E716
:100D4000002323B9BD46BDE8F0870123F9E74FF43E
:100D50008A7104FB01F1E031884B19440A3100F03B
:100D6000D9FC0028EED1854B4FF48A7202FB043483
:100D7000012384F8E83001F0CDFDD4F8E030C31A47
:100D8000192B05D940F6B832934202D9134600E038
:100D900019237A4AD2ED007AF8EE677A9FED787AD5
:100DA00027EE877A07EE903AF8EE677ADFED756AFC
:100DB00067EEA67A77EE277AFCEEE77AC2ED007A44
:100DC0003CE013464FF48A7202FB0535002385F898
:100DD000E830C5F8E030C546684B5B689B0A0133D4
:100DE000694A1381AEE7002042F8040B013B002B57
:100DF000F9DA2246304600F07FFA604B5B68002B40
:100E00004BD05E4B93F8D20000F02AFA82460028BD
:100E100047D05A4BD3F8D430002B4ED0574BD3F891
:100E2000D430234453454ED85FFA89F23146534BB0
:100E3000586800F07FFA00284CD1C5464F4B93F814
:100E4000D9504FF48A7202FB053393F8E830002B37
:100E5000C2D0E846494A4FF48A7303FB0523D3F80E
:100E6000E41053689942ACD144494FF48A7305FBAE
:100E700003F3CA18B2F8EC40E21C4FEA9209E033DF
:100E800019440E314A4609F1FF3392000732D20865
:100E9000A8EBC20295466E46A9E7012000F0D2F900
:100EA000AFE70024354B1C7200F000FA204600F03A
:100EB000C9F9354B0B221A818DE7304B93F8D200DC
:100EC000FFF7C4FCAAE72D4B93F8D2000130FFF7DF
:100ED000BDFCA9E7294B5A6822445A60D3F8D46074
:100EE0002644C3F8D46093F8D20000F0B9F98642E2
:100EF0000BD3224B93F8D220013283F8D220D3F8BF
:100F0000D420A2EB0A02C3F8D420FF2C23D91B4C17
:100F10004FF48A7303FB0545002385F8E830C5F8D4
:100F2000E030D5F8E43003F58063C5F8E43094F898
:100F3000D900FFF7B5FCFFF793FE94F8D9300133E1
:100F40005A4203F0030302F0030258BF534284F8ED
:100F5000D930C54672E70024084B1C7200F0A6F990
:100F6000204600F06FF900F0FBFC074A108108B141
:100F7000C546E7E6FFF778FAFAE77047B044002085
:100F80006666663FCDCCCC3D8C23002038B5054647
:100F90000C4602F067F950B1E38A282B1CD014D814
:100FA000012B0FD121462846FFF774FB0CE0237E6E
:100FB000022B09D1E38A012B06D121462846FFF7EF
:100FC00027FB01E0052B0CD038BD302BFCD121468E
:100FD0002846FFF79BFEF7E721462846FFF7D8FB98
:100FE000F2E7BFF34F8F0549CA6802F4E062044B91
:100FF0001343CB60BFF34F8F00BFFDE700ED00E070
:101000000400FA05014B1870704700BF98230020B8
:1010100030B585B04FF000531A68324B9A420FD06A
:1010200003F056FB044678B32F4A136C43F0007369
:1010300013642E4B9A6D2E4B9A4228D0002423E045
:101040004FF00054607DFFF7DDFF227D294B1A72BF
:10105000002309E01902274A4FF48A7000FB03229B
:10106000C2F8E4100133DBB2032BF3D94FF0005484
:10107000C92204F11601204800F03EF9E0220021C7
:10108000204600F04DF90124204605B030BD174B35
:101090001B6E23B37F2B01D90024F5E7174A01AB60
:1010A00010685168926807C3032101A800F088FB0B
:1010B0000E4B5B6D984201D00024E5E70B4B1B6D96
:1010C000994201D00024DFE7084D0023AB6595F875
:1010D0006000FFF797FFEA6D094B1A60D4E7002420
:1010E000D2E700BF9AAD44C5003802400066004018
:1010F0005041A0B0B0440020B944002058660040E0
:101100001023002030B583B000F02AFC1D4B18815D
:1011100002225A71002474B941F2D80304FB03F38C
:1011200019481A5855680122184909681844A847EF
:101130000134E4B2EFE700230193154B0093154B04
:101140004FF480521449154802F068F8144B19788E
:1011500099B901F0DFFB04464FF4C870FFF7E8F9D6
:10116000044404F516740F4B1C6003F0A7FA10B189
:10117000044B0F221A8103B030BD084802F06AF810
:10118000E7E700BF8C230020D83300201023002085
:10119000690500088D0F00089C230020A43300205F
:1011A00098230020A033002008B50CE0114B1860F4
:1011B00001F0B4FBFFF7F0FC13E0C82002F0BAFE28
:1011C0000D4B1B7AA3B1FFF74BFDFFF7F1FBFFF7C8
:1011D00065FC01F09FFB074B1B68C31AB3F57A7FD0
:1011E000E4D2054B1B7A002BE7D0FFF7B1FBE4E715
:1011F00008BD00BFE0490020B044002008B54FF60C
:10120000FF710120FFF7E4FC08BD00BF10B503F03B
:10121000C3F80A4B1880002406E003F093F8044456
:10122000074A136801331360B4F5803F05D2034BBE
:101230001B88034A10688342EFD810BD144A00206F
:10124000E849002008B503F001F908BD08B592008F
:1012500000F1006000F5803003F0F4F808BD00BF35
:1012600008B5064B1B88064A12689B1A834201D8B0
:10127000002008BD104403F065F8FAE7144A002086
:10128000E849002008B5034B1B68184403F086F8B2
:1012900008BD00BFE849002008B5034B1B6818448F
:1012A00003F094F808BD00BFE849002008B5074BDB
:1012B00093F824300BB9012008BD0449002381F8BC
:1012C00024300822086AFFF7C1FFF5E7EC49002047
:1012D000022800D07047024B4FF080529A61F9E724
:1012E00000080240022800D07047024B4FF48052A1
:1012F0009A61F9E700080240002304E011F803C0F6
:1013000000F803C001339342F8D37047034600202E
:1013100000E0013013F9012B002AFAD1704700BF19
:10132000034602E003F8011B624602F1FF3C002A7B
:10133000F8D170472DE9F843814688461546214B80
:1013400093F8243033B31F4A126A02EB83038342BB
:1013500020D0FFF7ABFF0346E0B930E0194E96F816
:101360002400C0F10804AC4228BF2C46E4B2A70018
:101370003A46414606EB8000FFF7BEFFB944B84449
:101380002D1BEDB296F824301C44E4B286F82440BC
:10139000082C0DD095B10B4B93F82430002BDDD1E8
:1013A0000848C0F820902022FF21FFF7B9FFD5E7B9
:1013B000FFF77CFF03460028ECD100E0012318462C
:1013C000BDE8F883EC4900202DE9F84380460E463D
:1013D000914640F2791200213046FFF7A1FF4346C3
:1013E00020220021304602F077F908F1040302229E
:1013F0002021304602F070F908F105030322222172
:10140000304602F069F908F106030322252130462F
:1014100002F062F908F1080310222821304602F098
:101420005BF908F1100308223821304602F054F924
:1014300008F1110308224021304602F04DF908F16D
:10144000120308224821304602F046F908F114033D
:1014500020225021304602F03FF908F118034022C3
:101460007021304602F038F908F120073B46082287
:10147000B021304602F030F908F121030822B821EA
:10148000304602F029F9C025002408E03B19023358
:1014900008222946304602F01FF9083501340F2C86
:1014A000F4D907F1120308222946304602F014F954
:1014B00005F108040025BB7C9D420BD205F1100309
:1014C0003B44033308222146304602F005F9083434
:1014D0000135F0E7B9F1000F10D0002598F832314E
:1014E0009D4214D205F598734344033308222146E4
:1014F000304602F0F1F808340135EFE708F599734A
:1015000007222146304602F0E7F80734E5E7E01D00
:10151000C008BDE8F88300BF38B505460C46002179
:101520002160C4F8031003462022204602F0D4F8BC
:101530002B1D02222021204602F0CEF86B1D032233
:101540002221204602F0C8F8AB1D032225212046A7
:1015500002F0C2F805F1080310222821204602F00B
:10156000BBF8072038BD00BFF0B583B007460E4674
:10157000047F009100230722194601F0ABFF731C82
:101580000093002301220721384601F0A3FF3CB15C
:10159000BB8ADB00083BDB08B3700825002414E09D
:1015A000B31C0093002305220821384601F092FF66
:1015B0000D25F3E73319033300930023082229464E
:1015C000384601F087FF08350134B3789C42F1D3E7
:1015D0000735ED083B7F2BB1B88A401B18BF0120AF
:1015E00003B0F0BDB88AA8422CBF00200120F7E765
:1015F000F0B583B007460C46057F00910023082212
:10160000194601F067FF661C3DB1BB8ADB00083B51
:10161000DB0863700825002413E0009600230822ED
:101620001146384601F056FF1025F4E7331901330F
:101630000093002308222946384601F04BFF083565
:10164000013433789C42F1D30735ED083B7F2BB151
:10165000B88A401B18BF012003B0F0BDB88AA84269
:101660002CBF00200120F7E7F8B506460F461446C8
:10167000812200213846FFF753FE3346082200211D
:10168000384602F029F814B10825002410E0731C34
:1016900007220821384602F01FF80F25F5E7331915
:1016A000023308222946384602F016F8083501347C
:1016B00073789C42F3D3E81DC008F8BDF8B5064620
:1016C0000F461446CE2200213846FFF729FE334646
:1016D00028220021384601F0FFFF083614B12825E2
:1016E000002410E0334608222821384601F0F4FF98
:1016F0003025F5E73319013308222946384601F031
:10170000EBFF0835013433789C42F3D3E81DC00861
:10171000F8BD00BFF0B583B007460E46047F0091C8
:1017200001231022002101F0D5FE3CB1BB8ADB0071
:10173000103BDB0873801025002414E0B31C0093D9
:10174000002309221021384601F0C4FE1925F3E7D1
:10175000331904330093002308222946384601F048
:10176000B9FE0835013473889C42F1D30735ED0882
:101770003B7F2BB1B88A401B18BF012003B0F0BDDE
:10178000B88AA8422CBF00200120F7E700B58E469A
:101790000AE040F3000C09490CEA010181EA50001B
:1017A0000133DBB2072BF4D91346013A23B11EF8FB
:1017B000013B58400023F5E75DF804FB2083B8EDBA
:1017C00030B583B004460B464FF0FF30014620E0B1
:1017D000001849410133DBB2072B0BD80029F7DA97
:1017E00010EB000C41EB010210488CEA000010499C
:1017F0005140EFE70EF1010E5FFA8EFEBEF1030FCE
:1018000006D801AB13F80E3081EA03610023E3E749
:101810002B465D1EADB22BB154F8043B01934FF043
:10182000000EEBE7C043C94303B030BD9336EAA9CD
:10183000EBE1F042F0B583B01F4B6A4693E803003A
:1018400082E8030008231D491D4803F0DFFA30B386
:1018500004460369B3F5702F23D8418B40F26E42E2
:10186000914220D100F11807164A024402F11001FA
:101870008B421BD39B1AA3F1100511490020FFF7DF
:1018800085FF06462A4639460020FFF77FFFA368FA
:10189000B3420DD1E36883420CD1002004E00A205A
:1018A00002E00B2000E00C2003B0F0BD1020FBE7AD
:1018B0000D20F9E70D20F7E7F84E0008DCFF0E00D9
:1018C000000001080800FFF7F0B583B0204B6A461E
:1018D00093E8030082E8030008231E491E4803F032
:1018E00095FA38B304460369B3F5702F24D8B0F8DD
:1018F000661040F26E42914220D100F16407174A0F
:10190000024402F15C018B421BD39B1AA3F15C05DC
:1019100011490020FFF73AFF06462A4639460020C3
:10192000FFF734FFA368B3420DD1E36883420CD1C3
:10193000002004E00A2002E00B2000E00C2003B0AD
:10194000F0BD1020FBE70D20F9E70D20F7E700BF01
:10195000044F000890FF0E00000001080800FFF788
:1019600010B5FFF767FF044608B9204610BDFFF722
:10197000ABFF0028F9D10446F7E700BF10B50446D5
:10198000037C0BB1204610BD006803F027FAF9E78D
:10199000BFF35B8FC368BFF35B8FBFF35B8F82685E
:1019A000BFF35B8F9A4208D94268BFF35B8F8068B0
:1019B000BFF35B8F101A18447047BFF35B8F8068CA
:1019C000BFF35B8F181A7047BFF35B8F0023C360B0
:1019D000BFF35B8FBFF35B8F8360BFF35B8F704799
:1019E0000346406800B97047BFF35B8F9A68BFF346
:1019F0005B8FBFF35B8FD968BFF35B8F914209D3D5
:101A00005868BFF35B8FDB68BFF35B8FD21A013A74
:101A10001044E8E70020F4E738B505460C46FFF728
:101A2000B7FFA04201D2002038BDBFF35B8FA96889
:101A3000BFF35B8F0C446968B4FBF1F301FB134403
:101A4000BFF35B8FAC60BFF35B8F0120ECE700BF9F
:101A500070B504460E461546FFF7C2FFA84200D3F4
:101A6000284608B9002070BD2368BFF35B8FE26889
:101A7000BFF35B8F134433606268BFF35B8FE3682F
:101A8000BFF35B8FD11A884207D971602168B160BA
:101A90009B1A1844F0600220E5E770600120E2E73D
:101AA00038B505460C46FFF79BFFA04201D2002047
:101AB00038BDBFF35B8FE968BFF35B8F0C44696887
:101AC000B4FBF1F301FB1344BFF35B8FEC60BFF396
:101AD0005B8F0120ECE700BF2DE9F04385B0814624
:101AE00088466946FFF7B4FF0746002425460EE006
:101AF00004AB03EBC40656F80C2C08EB050156F8B2
:101B0000100CFFF7F9FB56F80C3C1D440134A742BA
:101B1000EEDC29464846FFF7C3FF284605B0BDE87E
:101B2000F08300BFBFF35B8FC368BFF35B8FBFF36E
:101B30005B8F8268BFF35B8F9A4210D94368BFF313
:101B40005B8F8268BFF35B8F9B1A0B6073B1036876
:101B5000BFF35B8F8068BFF35B8F18447047BFF3A0
:101B60005B8F8268BFF35B8F9B1AEEE700207047A4
:101B7000F0B583B007460E461546FFF709FF044649
:101B80000190A84200D32C4614B9002003B0F0BD48
:101B900001A93846FFF7C6FF019B6BB1A34200D9EC
:101BA0000194306001987060A0420DD23B68B36030
:101BB000241AF4600220E9E73B6833607460002374
:101BC000B360F3600120E1E70120DFE72DE9F04198
:101BD00084B088466946FFF7CBFF074600242546B8
:101BE0000EE004AB03EBC40656F80C2C56F8101CA0
:101BF00008EB0500FFF780FB56F80C3C1D44013450
:101C0000A742EEDC284604B0BDE8F08138B50546B1
:101C1000FFF7DCFF044601462846FFF7FDFE20469D
:101C200038BD00BF10B5026854681A46A04710BD01
:101C30000020704700207047704700BF00207047A9
:101C40000E20704700F5805090F8C800C0F34000A7
:101C5000704700BF00F5805090F9D000704700BF7A
:101C600000F58050C0F8CC1001207047F0B583B06B
:101C7000BDF820500C6814F0005F40F089800C7BA8
:101C8000082C00F28880302484F311884469A66807
:101C900016F0806F0ED1A66816F0006F6BD1A668A3
:101CA00016F0805F02D04FF0020E05E0002080F3B6
:101CB00011885EE04FF0000EF4460E68002E5DDBEA
:101CC00076050EF1180E4FEA0E1E44F80E600E68EF
:101CD00016F0804F06D00CF118063601A75947F0D0
:101CE0000207A7510F7B0CF118064FEA061E04EB02
:101CF000061677608E6804EB0C17C7F88C614E6887
:101D0000C7F8886154F80E6046F0010644F80E608A
:101D100041F2680E0EEB4C14044400EB4C16764472
:101D200032607360D1F800E04F688E68C4F808E054
:101D3000E76026618E89A6820CF1840C00EB4C1CB6
:101D40009CF8044065F300048CF80440C5F3400699
:101D5000E4B266F341048CF80440E4B26FF3C304C8
:101D60008CF80440002484F31188009500F00CFEE8
:101D7000012003B0F0BD4FF0010E9DE7F60046F0E4
:101D800004060EF1180E4FEA0E1E44F80E609EE790
:101D90004FF0FF30EDE74FF0FF30EAE708B53023B2
:101DA00083F3118800F58050C06DFFF70DFE00230E
:101DB00083F3118808BD00BF70B504460D4641F29B
:101DC0005C068059FFF70CFE1F2801D8002070BD6B
:101DD00020222946A059FFF77FFE202814BF0020AB
:101DE0000120F4E72DE9F04188B006460D4617467C
:101DF0009846302383F3118800220023CDE9002385
:101E00000024ADF8084003948DF818408DF819406F
:101E10000494059441F25C040059FFF7B9FD1F28B2
:101E200006D8002070B980F3118808B0BDE8F081B1
:101E3000202269463059FFF7E9FE202814BF002010
:101E40000120EFE703AB07CB28606960AA601B881D
:101E5000AB81DDE90023C7E90023BDF80830A8F80D
:101E60000030002383F3118843463A462946304622
:101E700000F062FDD9E700BF10B5374B03600023C7
:101E8000436083600246354C42F8184B83611373FC
:101E90005373C36103629FED2E7B80ED0A7B038643
:101EA000436380F8403080F841308363C36300F1BE
:101EB000480423464FF07F0C0DE09FED257B83ED1A
:101EC000007B00221A81DA601A765A761A615A610A
:101ED00020330CF1FF3CBCF1000FEEDA00F582522A
:101EE000083200F580539C644FF48054DC64002475
:101EF0001C655C654FF0010C83F858C0DA6583F807
:101F000060C000F5835308334FF0020EBEF1000F9E
:101F100011DB9C469FED0E7BACEC027B00229A60AD
:101F20008CF80C208CF80D20DA601A619A6120334D
:101F30000EF1FF3EEAE700F5805383F8D01011B9A7
:101F4000074B436110BD074800F0DEFCAFF3008093
:101F50000000000000000000804F0008384F00081B
:101F600000640040104F000810B50446034B197878
:101F70004A1C1A70FFF780FF204610BD1C4A002043
:101F8000002977D070B582B00C46424B994211D9E6
:101F90000A234149B1FBF4FC013BDBB29E46581CCD
:101FA000BCFBF0F100FB11C131B1022B64D9013B44
:101FB000DBB2F3E71123ECE7BCFBF0F0411EB1F517
:101FC000806F5CD2C3EBC30E1EF103014DD4C1F38D
:101FD000C70C8DF800C0A3EB0C05EDB28DF80150D5
:101FE0000CF101064FF47A710CFB0111354491FBA1
:101FF000F5F189B2ADF80210B1F5617F18D9BEF1E3
:10200000010E34D4CEF3C70E8DF804E0A3EB0E031B
:10201000DBB28DF805300EF101054FF47A710EFB3D
:1020200001112B4491FBF3F3ADF80630019B0093B3
:102030009DF800104B1C9DF80160334400FB03F336
:10204000154DB5FBF3F3A3421BD10139C9B20F29DA
:1020500019D8D6B1082E1AD80138108000239370F1
:10206000D170013E1671012007E00731AFE70EF194
:10207000070EC7E700207047002002B070BD0020A7
:10208000FBE70020F9E70020F7E70020F5E7002054
:10209000F3E700BF3F420F0080DE800270B50646C6
:1020A0000D460024B4F57A7F0BD273695B6803F0A8
:1020B0000103AB4207D04FF47A7001F03BFF0134CB
:1020C000F0E7002000E0012070BD00BF032964D8C4
:1020D00070B588B004460D46164600F5805393F857
:1020E000C830C3F3800113F0040F00D1114604F58A
:1020F000805393F8C82061F3820283F8C82041F22C
:10210000680303EB451304EB030C05F1840304EBB4
:1021100043131B7913F0010F08D03EB105F184037E
:1021200004EB43131B7913F0080F10D06EB105F1C7
:10213000840304EB43131B7913F0080F05D1843596
:1021400004EB451443F00803237108B070BD00226E
:102150000023CDE900230023ADF8083003938DF868
:1021600018308DF819300493059303ABDCF80800A0
:10217000DCF80C10DCF8102007C3BCF814201A801F
:10218000DDE90C23CDE900230123ADF808302368F5
:10219000DB6B694620469847C8E7704742699369F8
:1021A00013F0700F23D00023936100E00133022B62
:1021B0001DDC03F1840200EB4212127912F0040FCD
:1021C000F4D003F1840200EB4212127912F0020FF4
:1021D000ECD04269064951F82310916003F1840262
:1021E00000EB4212117941F004011171DEE77047F2
:1021F000244F000870B582B0044616461D46436958
:102200009A6812F0010F16D163699A6812F4807F00
:102210001CD163699A6812F4803F24D104F580537D
:10222000D3F8CC0010B103681B6998472046FFF72C
:10223000B5FF02B070BD9A680121996000960195C2
:10224000C2F340020021FFF741FFDDE79A684FF437
:102250008071996000960195C2F3402201212046C9
:10226000FFF734FFD5E79A684FF480319960009604
:102270000195C2F3404202212046FFF727FFCDE738
:1022800038B504460846002977D1616901F10C0C84
:10229000DCF8001011F0030F6ED0DCF8001061695B
:1022A00000F11B052D014D5915F0040F69D100F106
:1022B0001B052D014D596D0DA56100F11B052D016B
:1022C0004D5915F0020F03D0A56945F08045A56171
:1022D00000F11B0501EB05156D6805F00F0E84F884
:1022E00024E001EB0011D1F8B8012077D1F8B80152
:1022F000000A6077D1F8B801000CA077D1F8B801D6
:10230000000EE077D1F8BC0184F82000D1F8BC01C0
:10231000000A84F82100D1F8BC01000C84F82200E6
:10232000D1F8BC11090E84F823103821CCF8001024
:10233000A569E069216A6563A063E163A18CA4F8E3
:102340004010A262E362002323862368DB6B04F162
:1023500028012046984704F5805393F8C82042F09E
:10236000040283F8C820D3F8CC0010B103681B69BD
:1023700098472046FFF712FF38BD616901F1100C44
:1023800086E700F11B052D014D59ED08A56145F0CB
:102390000045A56191E700BF302181F3118800213C
:1023A000022936DC30B502E0013102292DDC01F1D1
:1023B000840C00EB4C1C9CF804C01CF0040FF3D1FF
:1023C00001F1840C00EB4C1C9CF804C01CF0100FB5
:1023D000EAD000EB411E41F2680C0EEB0C045EF8F3
:1023E0000C50646895429C41DED244690B4D55F80F
:1023F0002150A56001F1840C00EB4C1C9CF804E01A
:102400004EF0040E8CF804E0CEE7002383F311882D
:1024100030BD002383F31188704700BF244F0008AC
:1024200008B5302383F31188FFF7B8FE002383F348
:10243000118808BD43699B6803F0E053B3F1E05F86
:102440002BD070B505460E464BB3302383F311886D
:10245000002400E00134022C1ADC04F1840305EBB3
:1024600043131B7913F0080FF4D104F1840305EB37
:1024700043131B7913F0040FECD141F2700101EB0F
:1024800044112944304600F0BDFA0028E2D100E0B2
:102490000120002383F3118870BD012070470020C4
:1024A000FAE700BF08B5302383F3118800F58050A8
:1024B000C06DFFF76DFA002383F311881F288CBFCE
:1024C0000020012008BD00BFF8B507460E4614469F
:1024D0001D4600231370FFF7E5FF80F00103337002
:1024E00025B129463846FFF7A5FF2070F8BD00BF8B
:1024F000F8B504460D4616461F4600F00FFA024690
:102500000B46297809B9307860B12046FFF744FFBF
:102510002046FFF785FF3B46324629462046FFF717
:10252000D3FF0120F8BD00BF302383F311881B4B7C
:102530001A6C42F000721A641A6A42F000721A624F
:102540001A6A22F000721A62002383F3118800F5E0
:10255000805393F8C83013F0010F1ED110B5044614
:1025600001B910BD302383F311880321132001F03A
:10257000CFFB0321142001F0CBFB0321152001F038
:10258000C7FB04F5805494F8C83043F0010384F885
:10259000C830002383F31188E3E770470038024016
:1025A00000F5805393F8D030012B00F231812DE9F2
:1025B000F0418AB004460E461746974A52F8232047
:1025C000002A36D0E6602774934B1B68002B34D06A
:1025D00004F5805393F8D030012B06D18E4B186848
:1025E00003681B6B9847002836D001212046FFF76F
:1025F0009BFF302383F311886269136823F0020381
:1026000013606269136843F0010313606269002379
:10261000536183F3118801212046FFF73FFD0346F4
:1026200048BB62694FF40041116018460AB0BDE82A
:10263000F081794A42F82300C4E741F2D80002F061
:102640008DFB054610B10021FFF716FC724B1D6093
:10265000002DBDD10023E8E76F4D00212868FFF76A
:1026600063FF286803685B683A463146984703462B
:102670000028BAD1D9E704F58053D86DFFF7A4F943
:102680004FF000082BE0202200216846FEF748FEAC
:10269000002302938DF814308DF8153003930493C2
:1026A000069341F2680505EB481504EB050EEC4670
:1026B000BCE80F006051CEF80410CEF80820CEF828
:1026C0000C30BCE80700CEF81000CEF81410CEF89D
:1026D00018209CF800308EF81C3008F10108B8F181
:1026E000020FD0D904F5805393F8C8206FF382020B
:1026F00083F8C8200023ADF820308DF822308DF803
:1027000023308DF8243008AA31462046FFF738FCE4
:10271000034600286FD0636961221A609DF8223059
:102720001B0603F040739DF82320120402F470226C
:1027300013439DF82420120502F4E0021343BDF870
:102740002020C2F309021343022F59D000216269ED
:102750000B43D361636913225A616269136823F0E2
:102760000103136000212046FFF798FC0346002870
:1027700049D004F5805292F8D0209ABB6169D1F813
:10278000002242F00102C1F800226169D1F8002262
:1027900022F47C5222F00E02C1F800226169D1F8C5
:1027A000002242F46062C1F8002261690022C1F88F
:1027B00014226169C1F80422616941F6FF70C1F811
:1027C0000C026169C1F840226169C1F84422626962
:1027D0000121C2F81C126169D1F8002222F0010225
:1027E000C1F8002204F5805494F8C82042F0020297
:1027F00084F8C82019E762694FF40041116014E7BA
:102800004FF00041A3E762694FF4004111600CE70B
:1028100000231846704700BF184A002008B500F092
:102820007DF802460B4652EA030102D0013A43F119
:10283000FF330449086808B1FFF7DCFC01F03CFAFB
:1028400008BD00BF184A002008B500F067F802462E
:102850000B4652EA030102D0013A43F1FF33044927
:10286000086810B10021FFF70BFD01F025FA08BD43
:10287000184A002008B500F051F802460B4652EA0B
:10288000030102D0013A43F1FF330449086810B153
:102890000121FFF7F5FC01F00FFA08BD184A0020EE
:1028A00000B59BB0EFF3098168226846FEF724FD6E
:1028B000EFF30583014B9B6BFEE700BF00ED00E0EB
:1028C00000B59BB0EFF3098168226846FEF714FD5E
:1028D000EFF30583014B9B6BFEE700BF00ED00E0CB
:1028E00000B59BB0EFF3098168226846FEF704FD4E
:1028F000EFF30583014B5B6BFEE700BF00ED00E0EB
:10290000FEE700BFFEE700BF0FB408B5029801F074
:10291000C3FAFEE708B501F011FE08BD08B501F0E5
:10292000E7FD08BD00207047012070470020704778
:1029300000207047704700BF30B583B084460D4615
:10294000043003C802AA02E9030069B10C461B88DF
:1029500013F0040F08D1DCF800309B6B60469847F9
:102960002A46C1B20098A047012003B030BD00BF85
:1029700082B0EC468CE80600031D9CE8030083E867
:102980000500012002B0704770B58AB004460E46BB
:10299000031D93E803000AAB03E9030069B10D4688
:1029A000BDF8383013F0040F0AD123689B6B204622
:1029B00098473246C1B20898A84701200AB070BDB6
:1029C00000220023CDE900230023ADF80830039353
:1029D0008DF818308DF819300493059303AB3068E7
:1029E0007168B26807C3B2891A80FFF797FFCDE913
:1029F00000010423ADF808302368DB6B69462046EC
:102A00009847DAE7036823F0604C0A6822F06041D7
:102A1000D00FB0EBD37F0FD0002B08DB002A09DBEF
:102A20008C4513D08C452CBF0020012070474FEA05
:102A30009C4CF3E7890CF3E7C3F38073C2F3807017
:102A40008C4504D08C452CBF002001207047834268
:102A5000FCD1F7E7084670470846704708467047BC
:102A600008467047401A83B2002800DB704703F124
:102A7000200000B2FAE700BF03780133DBB2037035
:102A80001F2B01D900230370704700BF082818D9F5
:102A900009280BD00A280BD00B280BD00C280BD000
:102AA0000D280BD00E280BD0402070470C2070470B
:102AB000102070471420704718207047202070475E
:102AC00030207047082818D90C280BD910280BD9AA
:102AD00014280BD918280BD920280BD930280BD94A
:102AE0000F207047092070470A2070470B2070475D
:102AF0000C2070470D2070470E207047034621F0D0
:102B0000604C20F06042C00FB0EBD17F0FD00029A5
:102B100008DB002B09DB944513D094452CBF002023
:102B2000012070474FEA9C4CF3E7920CF3E7C1F3A6
:102B30008071C3F38070944504D094452CBF00206D
:102B4000012070478142FCD1F7E700BF2DE9F04139
:102B500007460D46D0F82480B8F1000F0CD0464649
:102B60004446A4B169686068FFF7C8FF30B92368BC
:102B700026465BB11C46F4E7796208E0A04502D026
:102B800035602C6003E02C607D6200E02560BDE8CC
:102B9000F08100BFC37DC3F38402013262F3860378
:102BA000C375C38A6FF30903C382C37D6FF3C71371
:102BB000C375704738B504460D46006A04E00168E5
:102BC00004F10C00FFF74AFF10B10369AB42F6D1E4
:102BD00038BD00BF2DE9F043079CCE0803EBD405B8
:102BE00001F0070304F007041A442AE003F0070881
:102BF00004F00707C646B84538BFBE46CEF1080EFA
:102C0000D11A8E4528BF8E464FF47F4C2CFA0EFC0D
:102C10005FFA8CFC4CFA07FCD90800EB060919F89E
:102C2000011001FA08F1F940C9B24FEAD40815F8C9
:102C3000087079400CEA01014F4005F808707344B0
:102C400074449342D2D1BDE8F08300BF2DE9F04F28
:102C500087B004900E4605920393838AB1EBC30FAD
:102C600080F084801146DA0031448A4204D2D2B224
:102C7000F3B2D21AD3B20593049BDB683BB3272E81
:102C800036D8C6F12803059A9A422ED35FFA86FBFE
:102C9000CBF1280B5FFA8BFB00230093039B5A4672
:102CA000314604988068FFF795FF5E44059BA3EBCF
:102CB0000B04E4B2049B9F8A07F10057053FFF0015
:102CC000D3F80C9028214B46B9461F4627E0049BB9
:102CD0001B69002BD3D100230093039B059A314637
:102CE00004988068FFF776FF33E0DDF814B0D3E78F
:102CF000059C4FF0000BDDE72546CDF800B0039BA7
:102D00002A46711A381DFFF765FF2E44AB445FFA5F
:102D10008BFB641BE4B2A9EB0A093F684146A7B1EB
:102D20009CB1CA46B9F1E00F28BF4FF0E00A0AEBA8
:102D300001084645EFD2A8EB06039C42DCD35FFABC
:102D400088F5F3B2ED1AEDB2D7E7049B186900B12C
:102D500024B9BDF9140007B0BDE8F08FCDF800B07C
:102D6000039B2246711AFFF735FFF2E70020F2E7D6
:102D7000002070470139002307E0C25C10F801C051
:102D800000F803C04254013301398B42F5D3704738
:102D900080EA0120002303E0400080B20133DBB26F
:102DA000072B09D810F4004FF6D0400080B280F411
:102DB000815080F00100F1E7704700BF70B5164602
:102DC0001D46002411E0C4F12003A4F1200C26FAD2
:102DD00004F105FA03F3194325FA0CFC41EA0C014E
:102DE000C9B2FFF7D5FF0834A4B23F2CEBD970BDB0
:102DF00038B50C4604E014F8011BFFF7C9FF2A465A
:102E0000551E002AF7D138BD38B5058C072D0BD9D2
:102E10000446D0E902234FF6FF70FFF7CFFF2A46A2
:102E2000E169FFF7E5FF38BD4FF6FF70FBE700BF34
:102E300010B4016100F1040C002305E001EB431420
:102E4000CCF80040A44601339A42F7D80023CCF8CE
:102E5000003002814381838103605DF8044B704739
:102E60000346406848B102685A605A89013292B2FA
:102E70005A8199898A4200D99A81704708B5FFF72B
:102E8000EFFF08B10023036008BD00BF2DE9F84F34
:102E90008246894616461F46CB8AC3F30903052B93
:102EA00034D018460024042B0BD8BAB2A24208D959
:102EB000315D09EB0302D17601339BB20134A4B238
:102EC000F1E7BBB2A34218D9B9F816B0CBF3090B9E
:102ED000ABF1050293083E49A1FB0313C3EBC30307
:102EE000A2EB83031FFA83F8D9F8041081B150468E
:102EF000FFF7B0FD054601231CE00344B9F8162096
:102F000063F30902A9F81620012055E00024DBE74D
:102F10005046FFF7B3FF054601465046FFF79CFDBC
:102F2000C9F80400002D49D04FF000082CE001330F
:102F30009BB215462A68002AF9D107EB0B02053A25
:102F400092082349A1FB021292B2013292B293423B
:102F50001AD2B8F1000F17D15046FFF78FFF286043
:102F600078B3054610E0325D05EB0C031A710CF1E5
:102F7000010C1FFA8CFC0134A4B2BCF11B0F01D868
:102F8000A142F0D8A14204D8B9B2A1420AD9C4469C
:102F9000F3E75046FFF772FF2860A8B105464FF0EF
:102FA0000008F1E7B9F81630C3F30902114461F3E0
:102FB0000903A9F816300120BDE8F88F6FF0020070
:102FC000FAE76FF00200F7E76FF00200F4E700BFE6
:102FD0002549922443680B6041604389013B43814A
:102FE000704700BFF8B506460D460EE006F10C042A
:102FF0002046FFF72FFD014607682046FFF7EAFF4E
:1030000039462046FFF728FD686069680029EDD140
:10301000EB8A6FF30903EB8200200021F8BD00BFAB
:1030200008B5FFF71DFF034628B100220260426089
:103030008260C2600261184608BD00BF2DE9F04FF2
:1030400083B001921D465B69002B00F08A808146A7
:103050008B462B8C1BB1EA69002A00F08580072B78
:1030600006D94FF0800A4FF000084446474664E016
:1030700009F10C00FFF7D4FF0446002877D02A8C12
:10308000E9690830FEF738F9288C013080B2FFF783
:1030900019FDFFF7FBFC431E9BB22B840133237405
:1030A0006B691B7803F01F032A8C43F0C003224492
:1030B00013724BF00043636021464846FFF746FD1C
:1030C0000127384603B0BDE8F08F002007E0EA6929
:1030D000125D33441A72013080B20134A4B2034647
:1030E000062802D82A8CA242F1D82B8CA34235D0D4
:1030F000013080B2FFF7E6FCFFF7C8FC013880B270
:103100004FEA4813DBB243EA0A0A6B691B7803F003
:103110001F034AEA030A331883F808A04BF0004360
:1031200073600130307431464846FFF70FFD0137B8
:103130003FB288F001084FF0000A2B8CA342C0D0A8
:1031400009F10C00FFF76CFF064698B1002CBCD1CA
:10315000019B03721B0A43720220C0E74FF0400A32
:10316000C6E76FF00107ACE76FF00107A9E76FF062
:103170000207A6E76FF00207A3E700BF30B589B0EA
:1031800004460D46202200216846FEF7C9F8049542
:103190002046FFF765FE8646A0B1EC46BCE80F006E
:1031A000CEF80000CEF80410CEF80820CEF80C308F
:1031B000BCE80F00CEF81000CEF81410CEF818209E
:1031C000CEF81C30704609B030BD00BF70B5044663
:1031D00000F10C063046FFF7D1FF054628B1216A01
:1031E0003046FFF73DFC28602562284670BD00BFD1
:1031F00038B504460D46036A1BB1FFF7DBFC38B156
:1032000038BD0C30FFF7BAFF0028F9D02062F7E78D
:1032100029462046FFF7DAFFF2E700BFF8B504467B
:103220000E4615461F4630220021FEF779F8A760AA
:10323000069B6360079BA3626A09B5F5001F01D373
:103240004FF6FF7292B2314604F10C00FFF7F0FD29
:10325000F8BD00BF037823B919B111F0800F00D178
:1032600001707047007870472DE9F84305460C4619
:10327000D1F81C90B9F1000F23D094F81880B8F160
:103280001F0F3BD82846FFF7EDFF0646F8B9228C02
:10329000072A36D8278A37F0030335D149464FF637
:1032A000FF70FFF7A5FD47F6FE7303405B0243EA9C
:1032B00008633F0207F440773B431E434FF6FF721B
:1032C0000EE00B8C002BD8D06FF001050FE0238AA5
:1032D0001B0243EA08631E432046FFF795FD0246A2
:1032E000234631462846FFF7A9FE051E02DC284684
:1032F000BDE8F8836069FFF7BFFBF8E76FF00105F1
:10330000F5E76FF00305F2E76FF00105EFE700BFA7
:1033100070B58AB0044616461D462822002168462C
:10332000FDF7FEFF02960395BDF83830ADF810307A
:103330000F9B05939DF840308DF81830119B079333
:10334000BDF84830ADF8203069462046FFF78CFFC5
:103350000AB070BD2DE9F04106460F461546D36907
:103360002BB395F81880B8F11F0F2AD83046FFF715
:1033700079FF48B32C8A240444EA08642B7844EA91
:10338000C33444EA0724044344F080042846FFF78A
:103390003BFD02462B4621463046FFF74FFE041EFA
:1033A00002DD2B78012B08D02046BDE8F081138C7C
:1033B000002BD6D06FF00104F6E76869FFF75CFBDD
:1033C000F2E76FF00104EFE76FF00304ECE700BFF2
:1033D000F0B58BB004460D4617461E462822002144
:1033E0006846FDF79DFF9DF84C30012B14BF00236C
:1033F00001238DF80030029703969DF84030ADF818
:103400001030119B05939DF848308DF81830149BAF
:103410000793BDF85430ADF820306A46294620465F
:10342000FFF798FF0BB0F0BD406A00B10430704761
:1034300008B5416A0B6843620C30FFF7CBFD08BD4D
:103440002DE9F041054616469846076A3C4619E0C4
:1034500021462846FFF7C6FD05F10C072B6A1968BF
:103460003846FFF7FBFA286221463846FFF7B2FDDF
:103470002C6A274606E0216805F10C00FFF7EEFAFA
:10348000274604460CB3A168E368711A68EB03038E
:103490000F4A8A424FF0000272EB0303EBD22B6A11
:1034A000A342D5D021462846FFF79CFD23683B6008
:1034B00005F10C0321461C461846FFF78BFD3968C1
:1034C0002046FFF7CBFA0446DCE7BDE8F08100BFF9
:1034D00080841E002DE9F04182B0089E002800F093
:1034E000E28014461D460746002E00F0DF80531E82
:1034F000DBB23F2B00F2DD80012A02D1002D40F02B
:10350000DB800023009301936B4622463846FFF789
:103510009DFB071E3BDD14F0070F0AD002AB03EB47
:10352000D40111F8083C624202F00702134101F88D
:10353000083C012C0BD0082C2DD9102C2ED9202C76
:103540002FD9402C00F2BB804FF0080800E0A046C5
:10355000FFF70EFC40BB9DB1B4EBC80F10D0082C98
:1035600027D89DF80020631E22FA03F313F0010F01
:1035700006D00123A3405B42DBB213438DF8003039
:10358000002D72D0082C5ED89DF90030337038467B
:1035900002B0BDE8F0814FF00108D9E74FF0020812
:1035A000D6E74FF00408D3E741466846FFF7E2FB51
:1035B000D1E7102C0FD8BDF80020631E22FA03F3C8
:1035C00013F0010FDCD00123A3405B429BB21343F5
:1035D000ADF80030D4E7202C0CD8009A631E22FAF4
:1035E00003F313F0010FCBD00123A3405B421A4336
:1035F0000092C5E73F2C65D8DDF800C0019A631E34
:10360000C4F12100A4F121012CFA03F302FA00F025
:10361000034322FA01F10B4313F0010FB0D0012351
:10362000A4F12001C4F1200003FA01F123FA00F013
:103630000143A3405B4261EB41014CEA03030A43AF
:10364000009301929CE7102C03D8BDF90030338021
:103650009DE7202C02D8009B336098E7402C34D89B
:10366000DDE90023C6E9002391E7012C05D0082CF1
:1036700007D89DF80030337089E79DF8003033702B
:1036800085E7102C03D8BDF8003033807FE7202C6D
:1036900002D8009B33607AE7402C19D8DDE900237B
:1036A000C6E9002373E76FF0010770E76FF00107C9
:1036B0006DE76FF001076AE76FF0010767E76FF0EA
:1036C000080764E76FF0080761E76FF008075EE737
:1036D0006FF008075BE700BFF0B585B005460E4602
:1036E000402A03D8144612B9012400E040240022E5
:1036F00002920392012C06D0082C22D81B788DF858
:103700000830012703E01B788DF808302746FFF7C3
:103710002FFB68BB14F0070F0AD004AB03EBD401F6
:1037200011F8083C624202F00702934001F8083C9D
:1037300000962B462246002102A8FFF74BFA05B05F
:10374000F0BD102C04D81B88ADF808300227DEE746
:10375000202C03D81B6802930427D8E7402C05D8F7
:10376000D3E90023CDE902230827D0E70027CEE7DD
:10377000394602A8FFF7FEFACCE700BF70B506464F
:103780000C4605E00D6806F10C00FFF723FCE56030
:10379000E1680029F6D10023E360A3602361A382DE
:1037A00070BD00BF10F0800F04D010F4004F03D0A4
:1037B00001207047022070470020704710B5044672
:1037C000FFF7F0FF022802D0C4F3074010BDC4F396
:1037D0000F2014F07F0FF9D100F00300F6E700BFCF
:1037E0002DE9F04F99B006460D4603920493D1F8A7
:1037F00000904846FFF7D6FF0746022800F0888071
:10380000C9F30628B9F1000F80F2028219F0C04F07
:1038100040F001822C7B002C00F00082022F05D0AA
:103820003046FFF71FFD404540F0FB81C9F30463BC
:10383000099309F07F0A4846FFF7C0FF0A9040EA63
:10384000074949EA8A4949EA4869013C2C4494F805
:10385000048000220023CDE916235FEAD8130293E7
:1038600059D07468CDF800A03B46024616A93046F0
:10387000A047002800F0D88149463046FFF7B8FC41
:103880000446002800F0D381A368E168039A0593F9
:10389000D01A0790049B069163EB0103089395F8F7
:1038A0000DC0CDF82CC094F81AC0CDF830C094F8F3
:1038B0001790C9F3840908F01F0B59464846FFF7D3
:1038C000D1F80D9049465846FFF7CCF86368059A41
:1038D000069952EA010C34D09D4A07998A424FF06A
:1038E0000002089972EB010C7CD30B9A0C998A4266
:1038F0001BD0984B079A93424FF00003089A9341CC
:1039000072D2029B002B71D00F2871DD002319E0C9
:103910004FF0000876E749463046FFF74BF904467A
:103920000028B1D16FF00C0085E1029A002AE0D0A6
:103930000D9A012A01DD012304E0002BD9D00123D7
:1039400000E00123002B55D16A7BA37E9A4240F010
:103950007181029B13B118F0400F66D1C8F3401378
:10396000E27DB3EBD21F40F06981C2F384039B4533
:1039700040F06781029B002B00F0908018F0400F10
:1039800040F08C802B7B032B40F25E81039BA36075
:10399000049BE360AF1D2B7B033BDBB23A46214621
:1039A00006F10C00FFF772FA00286DDB2B796A79BB
:1039B00043EA02232383DDE916234FF6FF70FFF766
:1039C000FDF9A0822A7B033AD2B23946FFF710FAFA
:1039D000A082E37DDA43C2F3C01262F3C713E3753A
:1039E000002028E10123ADE70023ABE70023A9E78E
:1039F0000123A7E7E37D68F38603E375DBB26FF38A
:103A0000C713E37521463046FFF7ECFA6B7BA376CC
:103A1000029B002B98D1E37DC3F38402013262F351
:103A20008603E3756FF00C0005E1039BA360049A25
:103A3000E260202200210EA8FDF772FC039B0E938A
:103A4000049A0F922B1D10932B7B013BDBB2ADF838
:103A50004C300A9BADF84E308DF850708DF851B057
:103A6000099B8DF852308DF853A096F82C3083F0D6
:103A700001038DF85430B3680EA9304698472046AC
:103A8000FFF788F80020D6E021463046FFF7AAFA73
:103A90002046FFF77FF86FF00200CCE0029B13B9DD
:103AA00018F0400F1ED095F80C9009F1FF395FFA1D
:103AB00089F9B4F81680C8F30908B8F1040F30D8B2
:103AC00043464FF00008042B54D8C84552D205EBAA
:103AD00008021179E218D176013308F101085FFA82
:103AE00088F8F0E72F1D2B7B013BDBB23A462146DD
:103AF00006F10C00FFF7CAF9002808DB2A7B013A1F
:103B0000D2B23946A08AFFF773F9A08261E7214655
:103B10003046FFF767FA2046FFF73CF86FF00200E7
:103B200089E0616806F10C00FEF794FF024608B1D7
:103B3000052304E04FF000081CE01C330A4611681E
:103B40000029FAD1A8EB03034FF000080EE000BFF4
:103B500080841E0040420F0005EB08010879D1184F
:103B60000871013308F101085FFA88F81B2B01D8AE
:103B7000C845F1D3039B0E93049B0F9304F11B03E1
:103B80001093616806F10C00FEF764FF1190C845C0
:103B900035D2A84408F104031293E38AC3F309035E
:103BA0009944ADF84C900A9BADF84E308DF85070AA
:103BB0008DF851B0099B8DF852308DF853A096F8CE
:103BC0002C3083F001038DF85430002363602A7B8E
:103BD000013A291DA08AFFF70BF9A082238B984296
:103BE0000FD00EA93046FFF7C9FD2046FEF7D2FFE1
:103BF000A28A238B9A4209D06FF010001BE00023A9
:103C0000CAE7B3680EA930469847EAE7002012E0F9
:103C10006FF009000FE06FF009000CE06FF0090091
:103C200009E06FF00A0006E06FF00B0003E06FF0B0
:103C3000020000E0002019B0BDE8F08F6FF00D0029
:103C4000F9E76FF00E00F6E76FF00F00F3E700BF43
:103C5000EFF30983683305494A6B22F001024A6396
:103C600083F30988002383F31188704700EF00E095
:103C7000302080F3118862B60C4BD96821F4E061E2
:103C80000904090C0A4A0A43DA60D3F8FC2042F01E
:103C90008072C3F8FC2007490A6842F001020A60FA
:103CA0002022DA7783F82200704700BF00ED00E0A1
:103CB0000003FA05001000E0302383F31188104B55
:103CC0005B6813F4006F03D1002383F311887047FE
:103CD00010B5F1EE103AEFF30984683C4FF08073B1
:103CE000E361084BDB6B236684F3098800F096F8E8
:103CF00010B1054BA36110BD044BA361FBE700BFEE
:103D000000ED00E000EF00E03F0300084203000880
:103D10000901C9B2074A131883F8001300F01F0104
:103D2000400901238B4000F1600142F8213042F844
:103D30002030704700E100E00023037503691B6831
:103D4000996882689142FAD203605A6842601060B2
:103D50005860704708B50846302383F311880B7DFF
:103D6000032B0ED0042B10D043B14FF0FF338361EF
:103D7000FFF7E2FF002383F3118808BD83F3118866
:103D8000FBE78B6900221A60EFE74A680B68136053
:103D90004A685A60E9E700BF0023037503691B689E
:103DA000996882689142FAD803605A68426010604C
:103DB0005860704708B5FFF7BFFF08BD08B5064B50
:103DC000D9680875186802681A6053600122027584
:103DD000D860FCF79FFA08BD284A002030B587B0AC
:103DE00004460C4BDD68B1F1FF3F0FD02B460A4A69
:103DF000684600F01BF92046FFF7E0FF009B13B177
:103E0000684600F021F9A86907B030BDFFF7D6FF7A
:103E1000F9E700BF284A0020553D0008044BDA6846
:103E20001B6898689368984294BF002001207047EF
:103E3000284A002010B5084BD8681C6822681A6010
:103E4000536001222275DC60FFF7A6FF0146204681
:103E5000FCF760FA10BD00BF284A002008B50B4BE4
:103E600001221A70002353B109490A4800F074FC7A
:103E7000064B02221A70002383F3118808BD034AFF
:103E800002EB8302002151600133ECE7904C0020EB
:103E9000C44F0008284A002008B572B6044B1865C4
:103EA00000F0EEFA00F0D2FB024B03221A70FEE79C
:103EB000284A0020904C002008B500F0FFF808BD0B
:103EC0008B6002230B7500234B7508610846704711
:103ED00008B58168A1F1840341F8143C026941F8F6
:103EE000442C426941F8402C044A41F8242CC36810
:103EF000026820390248FFF7E3FF08BD2D030008E0
:103F0000284A002008B5FFF7E3FFFFF753FF08BD7D
:103F100008B5034BDB6898610F20FFF74FFF08BD22
:103F2000284A002008B5302383F31188FFF7F0FFFB
:103F300008BD00BF08B50146302383F3118808206F
:103F4000FFF74CFF002383F3118808BDF8B5154631
:103F50001C46C2608B60486003680B60596001605A
:103F6000092C00D80A24C068204400F0E1FB0A278D
:103F700000F0DAFB0646431B9C4202D90A2F07D801
:103F8000F8BD7C1C281900F0E1FB27463546EFE719
:103F9000012000F021FCF3E770B504460D46092925
:103FA00000D80A250A26601900F0D0FB00F0BCFBFF
:103FB000041BA54202D90A2E04D870BD013635462D
:103FC0000446F0E7012000F007FCF6E7F8B50546E7
:103FD0000E46174600F0A8FB2B689D4209D0EC68FE
:103FE000041B3C1900D33C469B68A34208D82B68AD
:103FF0000CE03B46024631462846FFF7A7FF14E097
:104000003946FFF7C9FFF2E7A41A1B689A68944281
:10401000FAD8B46033605A68726016605E609A685D
:10402000121B9A604FF0FF33AB60F8BD08B5036117
:10403000C260002343610A4601460248FFF7C6FFFB
:1040400008BD00BF384A002008B51B4B1B699842C9
:1040500010D042680368136042685A600268816841
:1040600093680B44936000230360134B4FF0FF32BF
:104070009A6108BD1968104A134643F8101F4B6037
:104080000021016012699A4212D0816893680B4442
:10409000936000F049FB084AD369A0EB030C126956
:1040A00091686145E5D91B1A1944FFF775FFE0E7F0
:1040B00000F046FBDDE700BF284A0020F8B50BE022
:1040C000002383F31188E368216920469847302351
:1040D00083F311886369CBB92C4D2C6900F024FB64
:1040E000EB69C21AA568954242D81D44274BDD6191
:1040F000616822680A60616851600022226053F89A
:10410000102F9A42DCD100F01BFBD9E700F00CFB2A
:104110000746461B6269B2420CD32B1A13441B4A52
:1041200052F8101F91420AD09E1900D23346174A06
:1041300012690CE0022000F04FFB0023EFE73A4643
:1041400021461348FFF702FF1FE05B1A12689168CF
:104150008B42FAD8A3602260516861600C605460A1
:104160009168CB1A9360094B4FF0FF329A61B3E725
:10417000064A52F8101F914207D0044AD0611B1A18
:10418000A1681944A160FFF707FFF8BD284A002085
:10419000384A002038B500F0C7FA054AD2E9084588
:1041A000031B181945F10001C2E9080138BD00BF21
:1041B000284A002000207047FEE700BF704700BF7C
:1041C0004FF0FF30704700BFBFF34F8F024BDB68EB
:1041D00013F4803FFAD17047003C0240014BF322B8
:1041E000DA607047003C024008B50B4B1B7803B106
:1041F00008BDFFF7E9FF094B1B69002B05DB074AE8
:10420000136823F480631360F2E7044B044A5A6096
:1042100002F188325A60F2E7984C0020003C0240DC
:104220002301674508B50C4B1B7803B108BDFFF7A8
:10423000CBFF0A4B1A6942F000421A611A6842F435
:1042400080521A601A6822F480521A601A6842F486
:1042500080621A60EAE700BF984C0020003C0240F0
:1042600012F0010F65D1F8B504460E461546131835
:10427000B3F1016F5FD8314B1B6813F0010F01D10F
:10428000002059E0FFF7B0FFFFF7A8FFFFF79CFF02
:10429000032D29D914F0030F26D1294A136923F4D9
:1042A00040731361136943F4007343F00103136116
:1042B00037682760BFF34F8FFFF786FF23689F4261
:1042C00003D1043D04360434E2E71D4A136923F0A8
:1042D0000103136104E01A4A136923F00103136117
:1042E000FFF7A0FF002027E0012D19D9144A136918
:1042F00023F440731361136943F4807343F00103A3
:10430000136133882380BFF34F8FFFF75DFF23884E
:104310009BB232889A42DED1023D02360234E3E794
:10432000074A136923F001031361FFF77BFF0120A4
:1043300002E0002070470020F8BD00BF00380240B6
:10434000003C0240014B53F820007047D04F00085A
:104350000B281AD870B506460D4B1B788BB9002474
:104360004FF0006508E00B4B43F824502046FFF760
:10437000E9FF05440134E4B20B2CF4D9044B0122CB
:104380001A70044B53F8260070BD0020704700BF20
:10439000CC4C00209C4C00200C2070470B2801D9ED
:1043A0000020704738B50546FFF7D2FF044628467F
:1043B000FFF7C8FF30B12368B3F1FF3F04D10438E1
:1043C0000434F7E7012038BD0020FCE70B2801D9B1
:1043D0000020704738B50446FFF7F6FEFFF704FFEC
:1043E000FFF7FCFE154BA3FB0423DB081A4603EB87
:1043F0004303A4EB8303DB00DBB2D201D2B213434D
:1044000043F4007343F002030D4A1361136943F44C
:1044100080331361FFF7D8FE2046FFF799FF05466A
:104420002046FFF78FFF0146284600F00BF9FFF703
:10443000F9FE2046FFF7B2FF38BD00BFABAAAAAA1B
:10444000003C024008B5FFF70BFF08BD08B5034666
:1044500010B10A4A127822B113B9084B1B7833B94C
:1044600008BDFFF7C1FE054B01221A70F8E7034BA8
:1044700000221A70FFF7D6FEF2E700BF984C00202A
:1044800010B500240BE0074804EB44039A001346E0
:1044900003445968805800F0D7F80134E4B2012C85
:1044A000F1D910BD0050000808B50846114600F0CB
:1044B00077FC08BD08B5012000F072FC08BD00BF04
:1044C00008B5084600F08AFC08BD00BF302383F31E
:1044D00011887047002383F311887047302383F3DA
:1044E00011887047002383F311887047FFF752BE8D
:1044F000EFF3118303BB00B583B0EFF30583C3F380
:10450000080363B9FFF7E2FFFFF7F0FFCDE9001002
:10451000FFF7E0FFDDE9001003B05DF804FBFFF7F3
:10452000DDFFFFF7E3FFCDE90010FFF7DBFFDDE97B
:10453000001003B05DF804FBFFF7D8BF38B5FFF7F4
:10454000D7FF114C114AC00840EA4170A0FB025E3F
:10455000C908A0FB040C1CEB050CA1FB04404FF0A8
:1045600000035B41A1FB02121CEB040C43EB0000B7
:1045700011EB0E0142F10002411842F1000009095D
:1045800041EA007038BD00BFCFF753E3A59BC420BC
:1045900009E000F1010C064A52F8202041F8042BF2
:1045A0001A465FFA8CF0531EDBB2002AF1D1704735
:1045B0005028004010B4124B1B6F13F4004F08D169
:1045C0000F4B1C6F44F400741C671C6F44F40044D0
:1045D0001C670C4C236843F48073236009E000F1EE
:1045E000010C51F8044B084A42F820401A465FFA81
:1045F0008CF0531EDBB2002AF1D15DF8044B7047FA
:1046000000380240007000405028004000B583B0E0
:10461000012201A90020FFF7BBFF019803B05DF85C
:1046200004FB00BF10B582B00446FFF7EFFFA042C5
:1046300001D102B010BD0194012201A90020FFF7B1
:10464000B9FFF6E7704700BF704700BF704700BF73
:10465000074B45F255521A6002225A6040F6FF722B
:104660009A604CF6CC421A60024B01221A707047D5
:1046700000300040D44C0020034B1B781BB1034B8F
:104680004AF6AA221A607047D44C0020003000403D
:10469000044B1B6823B9044BD3F87428014B1A60F0
:1046A000704700BFD04C002000300240024B4FF05A
:1046B0008072C3F8742870470030024008B5FFF7D5
:1046C000E7FF024B1868C0F3407008BDD04C0020D3
:1046D00008B5FFF7DDFF024B1868C0F3007008BD96
:1046E000D04C0020704700BFFEE700BF084B0949CF
:1046F00003E051F8042B43F8042B074A9342F8D304
:1047000002E0002243F8042B044A9342F9D3704795
:10471000604D0020A8510008604D0020604D002031
:1047200008B500F0DBF808BD4FF08043586A7047C9
:104730004FF08043586300221A610222DA6070470A
:104740004FF080430022DA60704700BF4FF0804393
:1047500058637047FEE700BF70B586B004460E464A
:10476000194B5860002585620163FFF781FA2460C8
:104770006460A560E56204F11003236163614FF09A
:10478000FF33A361E561FFF7CFFF02462B46C4E983
:104790000823256580230D4A04F134012046FFF7E4
:1047A0008FFBE06001230375094A00927268019251
:1047B000B26802920393074B049305956846FFF78E
:1047C000A1FB06B070BD00BF904C0020185000083F
:1047D0002050000855470008024AD36A0343D362B9
:1047E000704700BF284A00204B6843608B68836095
:1047F000CB68C3600B6943614B6903628B69436299
:104800000B680360704700BF10B5214B1A6940F276
:10481000FF110A431A611A6922F4FF7222F00102A1
:104820001A611A691A6B0A431A631A6D0A431A65E8
:104830001B6D184C21461848FFF7D6FF04F11C01E8
:104840001648FFF7D1FF04F138011548FFF7CCFFF8
:1048500004F154011348FFF7C7FF04F17001124837
:10486000FFF7C2FF04F18C011048FFF7BDFF04F110
:10487000A8010F48FFF7B8FF04F1C4010D48FFF786
:10488000B3FF04F1E0010C48FFF7AEFF10BD00BF1D
:104890000038024028500008000002400004024096
:1048A00000080240000C02400010024000140240C8
:1048B00000180240001C02400020024008B5FFF72B
:1048C000A3FF00F095F808BD08B500F025FAFFF742
:1048D000C5FAFFF7DDFE08BD704700BF0F4B1A6C2D
:1048E00042F001021A641A6E42F001021A661B6E4F
:1048F0000B4A936843F0010393604FF080435322C7
:104900009A624FF0FF32DA6200229A615A63DA60EB
:104910005A6001225A611A60704700BF0038024095
:10492000002004E008B54FF080421369D168C9B295
:104930000B40D943116113F0020F00D108BD3023A1
:1049400083F31188FFF7B8FA002383F31188F5E7A2
:104950000B4A136843F4807313600A4B1B6F03F414
:104960004073B3F5007F05D0064B4FF480321A67D1
:1049700000221A67024A536823F400735360704799
:10498000007000400038024008B5184B1A696FEA01
:10499000C2526FEAD2521A611A69C2F308021A614E
:1049A0001A695A694FF0FF3058615A6900215961FC
:1049B0005A691A6A62F080521A621A6A02F08052C8
:1049C0001A621A6A5A6A58625A6A59625A6A1A6CA0
:1049D00042F080521A641A6E42F080521A661B6EC0
:1049E000FFF7B6FF00F076F908BD00BF00380240BF
:1049F0003B4B4FF080521A643A4A4FF440411160E9
:104A00001A6842F001021A60354B1B6813F0020F5E
:104A1000FAD0334A936823F003039360304B9B68CA
:104A200013F00C0FFAD12E4B1A6802F0F9021A603B
:104A300000229A601A6842F480321A60284B1B6880
:104A400013F4003FFAD0264A536F43F00103536733
:104A5000234B5B6F13F0020FFAD0214B224A5A60AE
:104A60001A6842F080721A601E4B5B6813F4804F24
:104A7000FAD01B4B1B6813F0007FFAD0184B1B4A6F
:104A80009A601B4B1A681B4B9A421FD01A4B40F27C
:104A900005721A60184B1B6803F00F03052BF9D140
:104AA0000F4A936843F0020393600D4B9B6803F039
:104AB0000C03082BF9D10A4B5A6C42F480425A6419
:104AC0005A6E42F480425A665B6E70470B4B1A680E
:104AD0000B4B9A42DAD1084B40F205121A60D9E723
:104AE00000380240007000400854400700948838A5
:104AF000002004E011640020003C024000ED00E0D2
:104B000041C20F4108B5074A536903F001035361DD
:104B10002BB1054B1B6813B1034A50689847FFF748
:104B2000CBF808BD003C0140D84C002008B5074A2E
:104B3000536903F0020353612BB1054B9B6813B11A
:104B4000034AD0689847FFF7B7F808BD003C01401A
:104B5000D84C002008B5074A536903F00403536199
:104B60002BB1054B1B6913B1034A50699847FFF7F6
:104B7000A3F808BD003C0140D84C002008B5074A06
:104B8000536903F0080353612BB1054B9B6913B1C3
:104B9000034AD0699847FFF78FF808BD003C0140F1
:104BA000D84C002008B5074A536903F0100353613D
:104BB0002BB1054B1B6A13B1034A506A9847FFF7A4
:104BC0007BF808BD003C0140D84C002010B51A4BC2
:104BD0005C6904F478725A6114F0200F05D0174B09
:104BE0009B6A13B1154AD06A984714F0400F05D05C
:104BF000124B1B6B13B1114A506B984714F0800F86
:104C000005D00E4B9B6B13B10C4AD06B984714F434
:104C1000807F05D0094B1B6C13B1084A506C984734
:104C200014F4007F05D0054B9B6C13B1034AD06C84
:104C30009847FFF741F810BD003C0140D84C0020D8
:104C400010B51F4B5C6904F47C425A6114F4806F08
:104C500005D01C4B1B6D13B11A4A506D984714F4C4
:104C6000006F05D0174B9B6D13B1164AD06D984756
:104C700014F4805F05D0134B1B6E13B1114A506EB4
:104C8000984714F4005F05D00E4B9B6E13B10D4A8C
:104C9000D06E984714F4804F05D00A4B1B6F13B1A8
:104CA000084A506F984714F4004F05D0054B9B6F8E
:104CB00013B1044AD06F9847FEF7FEFF10BD00BF46
:104CC000003C0140D84C002008B5FFF72BFEFEF752
:104CD000F3FF08BD08B506210846FFF719F80621BD
:104CE0000720FFF715F806210820FFF711F8062125
:104CF0000920FFF70DF806210A20FFF709F8062121
:104D00001720FFF705F806212820FFF701F80721F3
:104D10001C20FEF7FDFF08BD08B5FFF735FE00F0CB
:104D200005F8FFF7D9FDFFF7FBFC08BD002307E0FE
:104D3000054A002142F8331002EBC30251600133EF
:104D40000F2BF5D9704700BFD84C00200B46014609
:104D5000184600F02DB8000000F040B8012838BF18
:104D6000012010B50446204600F030F830B900F0BC
:104D700007F808B900F00CF88047F4E710BD000010
:104D8000024B1868BFF35B8F704700BF584D00207F
:104D900008B5062000F084F80120FFF70DFA0000A6
:104DA000024B0A4601461868FFF77EBB1C23002011
:104DB00010B5054C13462CB10A4601460220AFF34C
:104DC000008010BD2046FCE700000000024B0146B9
:104DD0001868FFF76FBB00BF1C230020024B014681
:104DE0001868FFF76DBB00BF1C23002010B5013908
:104DF0000244904201D1002005E0037811F8014FF0
:104E0000A34201D0181B10BD0130F2E72DE9F0419B
:104E1000A3B1C91A17780144044603F1FF3C8C4240
:104E2000204601D9002009E00578BD4204F10104C3
:104E3000F5D10CEB0405D618A54201D1BDE8F081EF
:104E400015F8018D16F801EDF045F5D0E7E7000003
:104E50001F2938B504460D4604D9162303604FF0C8
:104E6000FF3038BD426C12B152F821304BB92046A8
:104E700000F030F82A4601462046BDE8384000F0F0
:104E800017B8012B0AD0591C03D116230360012047
:104E9000E7E7002442F82540284698470020E0E74D
:104EA000024B01461868FFF7D3BF00BF1C23002048
:104EB00038B5074D00230446084611462B60FFF71E
:104EC0007FF9431C02D12B6803B1236038BD00BFBA
:104ED0005C4D0020FFF76EB96F72672E61726475CA
:104EE00070696C6F742E41522D46343037536D61AA
:104EF000727442617400000040A2E4F1646891069B
:104F00000000000041A3E5F265699207000000007F
:104F10004261642043414E496661636520696E6465
:104F200065782E00800000000080000000008000F6
:104F30000000000000000000251C0008A12500085A
:104F4000F1240008611C00086D1C0008E51D000824
:104F5000311C0008411C0008351C00083D1C0008DD
:104F6000391C00089D1D0008451C00087129000817
:104F7000551C0008B91D00080000000000000000DA
:104F8000251C0008012900082529000829290008F6
:104F90008929000839290008311C00082D2900083A
:104FA000351C000831290008391C00083529000883
:104FB00001290008712900080129000801290008B9
:104FC00063300000C04F0008804A0020904C002051
:104FD00000400000004000000040000000400000D1
:104FE00000000100000002000000020000000200BA
:104FF00000000200000002000000020000000200A9
:105000000001002000FF010001000000000002205C
:1050100000000200020000006D61696E00000000E7
:1050200069646C65000000000000802A0000000038
:10503000AAAAAAAA00000024FFFF000000000000A6
:10504000009009000000000000000000AAAAAAAA1F
:1050500000000000FFFF0000000000000000000052
:105060000000000500000000AAAAAAA60000000097
:10507000FFEF000000000000000000000000000042
:1050800000000000AAAAAAAA00000000FFFF00007A
:105090000000000000000000000000000000000010
:1050A000AAAAAAAA00000000FFFF0000000000005A
:1050B000000000000000000000000000AAAAAAAA48
:1050C00000000000FFFF00000000000000000000E2
:1050D0000000000000000000AAAAAAAA0000000028
:1050E000FFFF0000000000000000000000000000C2
:1050F000000000000A0000000000000003000000A3
:10510000000000000000000000000000000000009F
:10511000000000000000000000000000000000008F
:1051200000000000000000006E040000000000000D
:1051300000000F000000000040420F00FE2A0100A6
:10514000D204000020230020000000000000000026
:10515000000000000000000000000000000000004F
:10516000000000000000000000000000000000003F
:10517000000000000000000000000000000000002F
:10518000000000000000000000000000000000001F
:10519000000000000000000000000000000000000F
:0851A000000000000000000007
:00000001FF
